:020000040000FA
:02000000B52821
:080008008C00030E8D00303066
:10001000840091018F0A031006180314800D910AC1
:100020009119840A9119910100000000061C2028F2
:10003000061C2028061C2028061C20288F032428A4
:100040000F08DE3E031D0A2838200038031D302823
:100050004A200038031D302885200038031D302831
:100060000E148F010D0E83008C0E0C0E8B100900E8
:100070000F08183C031D00343008403C031D0034B9
:100080003108033C031D00342030840041302C2112
:10009000970A01340F08083C031D00343008003C67
:1000A000031D00343030840009308000840A0030A1
:1000B0008000840A00308000840A08308000840AAE
:1000C0003030840019302C21203084000030800032
:1000D000840A80308000840A80308000840A803066
:1000E0008000840A80308000840A80308000840A86
:1000F00000308000840A00308000840A08308000CC
:10010000840A20308400413001340F08083C031D6C
:1001100000343008413C031D00343030840000308E
:100120008000840A80308000840A80308000840A45
:1001300080308000840A80308000840A8030800013
:10014000840A00308000840A00308000840A023073
:100150008000840A02308000840A08308000840A0B
:100160003030840051302C2101348316861406145B
:1001700005128611061106120113831206128F0151
:1001800005168B100B168B1386110615861C6E2117
:1001900003309600861CC62855213B3094003A3027
:1001A00095008618C628950BD128940BCF2831309E
:1001B0009400940BD928960BCA2897018B17061127
:1001C0008615E22817080A3C031CC32898019901E8
:1001D0004A21003C0319C3286E210616991386187C
:1001E0009917632198108618981463219811861C1A
:1001F0009815632119128618191663211812861C86
:100200001816632199118618991563211911861CF6
:100210001915632119108618191463219910861C69
:100220009914632118108618181463211811861C5C
:100230001815632119138618191763219912861C42
:10024000991663210612861CE22863211808A00073
:100250001908A1009701E22890009101000892007E
:10026000840A05120000910A920D031805169119CF
:100270004529000000000000000000000000000010
:1002800005169003031D3129080000089200840A16
:100290009101402953309400533095008618013461
:1002A000950B4E29940B4C2900344B3094004B3065
:1002B0009500950B5929940B57296A309400940B9B
:1002C0005F2900000800FF309400940B65299E30E0
:1002D0009400940B6929000000000800CE309400BF
:0A02E000940B7029000000000800D4
:02400E00FA3F77
:00000001FF
